:020000040800F2
:10000000A80B0020D5000008E1150008F514000831
:1000100000000000000000000000000000000000E0
:10002000000000000000000000000000B7190008F8
:100030000000000000000000B5190008B919000810
:100040000501000800000000050100080501000886
:100050000501000805010008050100080501000868
:100060000000000005010008050100080501000866
:100070000501000805010008050100080000000056
:100080000501000800000000000000000501000854
:100090000000000005010008050100080501000836
:1000A0000000000005010008000000000501000834
:1000B000050100080000000000000000C92400083D
:1000C0000348854600F05AF800480047112500080B
:1000D000A80B00200C4880F308880C480168090E22
:1000E0000B4A914205D10B480B4901600B480C4962
:1000F00001600C4880470C480047FEE7FEE7FEE73A
:10010000FEE7FEE7FEE70000A80B00200400000069
:100110001F00000018100240010000000000014014
:10012000000000001D1A0008C100000830B50B4691
:10013000014600202022012409E00D46D5409D42C1
:1001400005D31D469540491B254695404019154647
:10015000521E002DF1DC30BDD2B201E00270401C15
:10016000491EFBD270470022F6E710B513460A4637
:1001700004461946FFF7F0FF204610BD064C012546
:10018000064E05E0E36807CC2B430C3C984710343F
:10019000B442F7D3FFF798FF102600083026000876
:1001A00070B58C180578401C6B075B0F01D1037884
:1001B000401C2A1106D10278401C03E006780E701C
:1001C000401C491C5B1EF9D12B0705D40023521E8D
:1001D0000DD40B70491CFAE70378401CCB1A921C13
:1001E00003E01D780D70491C5B1C521EF9D5A1421D
:1001F000D8D3002070BD704731B500F0BBF8009C2B
:100200000546601C00D0641C00F0B4F8401BA042FE
:10021000FAD338BDF8B500238DE001249C40A446F4
:1002200022407DD04C68022C01D0122C0CD1DC086D
:10023000A40027183C6A5D07ED0E0F26AE40B443BC
:100240000E69AE4026433E6205685E000324B4405A
:100250000F79A543BF07BF0FB7402F4307604D6815
:10026000012D05D0022D03D0112D01D0122D0ED15C
:100270008568CF68A543B7402F43876047686546C8
:10028000AF430D79ED06ED0F9D403D434560C568D8
:10029000A5438C68B4402C43C4604C68E40049D545
:1002A000284CA56901263543A561A4699D08344001
:1002B0000094254CAD002F19BC689D072E0F0F250B
:1002C000B540AC430925ED06A84201D100250FE059
:1002D0001E4DA84201D101250AE01D4DA84201D1C1
:1002E000022505E01B4DA84201D1032500E00525AC
:1002F000B5402543BD60184C25684E689543F6030C
:1003000000D51543256065684E689543B60300D552
:1003100015436560A5684E689543F60202D500E076
:1003200008E01543A560E5684E689543B60200D520
:100330001543E5605B1C0A681446DC4000D06CE79E
:10034000F8BD000000100240000001400004004819
:1003500000080048000C0048000401400069084003
:1003600000D001207047002A01D08161704781626E
:1003700070470000014800687047000070000020CE
:1003800002480168491C01607047000070000020AD
:1003900010B506480168102211430160002000F0EA
:1003A00007F800F017F8002010BD00000020024000
:1003B00010B5044600F09AFE7D21C900FFF7B6FE95
:1003C00001F080F800222146501E00F027F800209E
:1003D00010BD000008B50A488169012211438161FE
:1003E000816911400091C26901040A43C261C06978
:1003F000084000900348016810221143016008BDC5
:100400000010024000000140C106C90E01208840D2
:10041000014908607047000000E100E010B501F0FC
:10042000E1F810BD10B50C0606D54906490E1C248E
:1004300061430818283004E01C2461430818FF3089
:10044000093099B2002A06D001228272C180190CAB
:100450000181002010BD002282728180F9E71C22F8
:100460004A43121810B5FF30FF300230926BC0695A
:1004700001F023FD10BD1C224A43121810B5FF30B5
:10048000FF32FF30013202309269C06901F070FD25
:1004900010BD0000F0B54B065B0E1C461C225343FA
:1004A000CD091A18002D01D0283201E0FF3209329F
:1004B00003461470C909FF335170E133197A0129D9
:1004C0003DD001211972947A4C49002C547838D0CF
:1004D000002C147805685FD0A4002E5B760404D548
:1004E0002E5B474F0E403E432E5314780568A40000
:1004F0002E5B760604D52E5B424F0E403E432E53B4
:1005000014780568A4002E5B0E403D490E432E531F
:10051000117806688D00715B384C30342140394CBD
:10052000403C21437153016810788200885A344D51
:10053000F13D28402043885200201872F0BD02206F
:10054000F0BD002C11D014780568A4002E5B76064F
:1005500004D52E5B0E402B490E432E5304681078B1
:100560008100605A254A303210E015780468AD00E9
:10057000665B760404D5665B0E4021490E436653E4
:10058000046810788100605A1D4AF13A10401D4AF3
:10059000403A10436052CFE7A4002E5B760404D5A6
:1005A0002E5B174F0E403E432E5314780568A4006F
:1005B0002E5B760604D52E5B124F0E403E432E5323
:1005C00014780568A4002E5B0E400E490E432E538E
:1005D000117806688D00715B094CF13C2140094C93
:1005E000403C21437153056810788100685A034AE2
:1005F00030321040204368529EE700008F8F000089
:1006000080C00000C0800000F0B54B06CA095B0E38
:10061000002A04D01C225A431218283204E01C225B
:100620004A431218FF3209320024947013700346B3
:10063000C909FF335170E133197A01291DD0012115
:10064000197251781B4E00291B4C1178056816D081
:1006500089006F5A7F0605D56F5A3740164E4036CF
:1006600037436F52117800688A00815A114D303536
:10067000294010256940202515E00220F0BD8900A1
:100680006F5A7F0404D56F5A37400C4E37436F5270
:10069000117800688A00815A084DF13D29400125F2
:1006A0002D0369406D00694021438152002018727A
:1006B000F0BD00008F8F00008080000080C000002F
:1006C000F0B54D066D0E2E461C246543CF092C183F
:1006D000002F01D0283401E0FF3409342670C90905
:1006E00061700146FF31E260E131E3708C46097AC6
:1006F00001290ED0012261460A72E378984A99498D
:10070000002B08D0012B7DD0022B0BD0032B19D14D
:1007100010E00220F0BD25780368AD005E5B164056
:10072000914A0DE0237805689B00EE5A16400E436F
:10073000EE5207E025780368AD005E5B16408B4AF9
:1007400016435E5325780668AB00F25A884F3A404C
:100750000A432A43F252A27A002A62D0227807681A
:1007600095007B5B824A834E134033437B53E3887F
:1007700050265D0803686D00F65AF6182378DF00EE
:1007800001239B02FB18F552238950265D0803685C
:100790006D00F65AF6182378DF00774BFB18F552F8
:1007A00063780768002B23787ED09B00FD5A6D0488
:1007B00004D5FD5A714E15403543FD522378076824
:1007C0009B00FD5A6D0605D5FD5A664E1540403614
:1007D0003543FD52237805689B00EE5A1640674A60
:1007E0001643EE522278036892009D5A604E3036CE
:1007F00035400D439D52026820788300D05A5F4CEB
:10080000F13C00E006E020400843D0520020614661
:100810000872F0BD25780368AD005E5B1640584A4B
:100820008EE76278002AA28821D0530802685025FA
:10083000AD5A5B00AD182278D60001229202B218A0
:10084000AB522278036892009D5A6D0606D59D5AD8
:10085000474E3540434E403635439D52026820781E
:100860008300D05A424C30342040202443E05308C7
:1008700002685025AD5A5B00AD182278D6003E4A7A
:10088000B218AB52026850239B5A3B4D9A182378FA
:10089000AD1CDB005B19D518E2683E2A0CD9D302E7
:1008A0001B0CD20603D100E027E05B1E9BB29A022C
:1008B0000123DB031A4306E0D3031B0CD20701D04C
:1008C0005B1C9BB29A022A80237802689B00D55A4F
:1008D0006D0405D5D55A264E3540284E3543D552A0
:1008E000026820788300D05A244CF13C2040012437
:1008F000240360406400604086E79B00FD5A6D045D
:1009000004D5FD5A1D4E15403543FD522378076826
:100910009B00FD5A6D0605D5FD5A124E1540403616
:100920003543FD52237805689B00EE5A16400D4A68
:1009300040321643EE52227805689300EA5A0F4E71
:10094000F13E3240012636037240760072400A437F
:10095000EA52026820788300D05A054C303450E7C0
:100960008F89000080800000808200008086000067
:100970008F8F0000808100000404000080C0000010
:1009800080840000F0B54D066D0E1C246C432418C5
:10099000FF340934636122610022A2616270257014
:1009A000E5681E46AB4201D92B46F21A6261A67A6F
:1009B00049060122890DD203002E2F4D06680CD066
:1009C0005027BF5BBE192F1FC91976183E2B15D9AA
:1009D000D902090CDF060CD00DE05027BF5B491986
:1009E000BE19751820E08902114300E089022980B0
:1009F00032E0491E89B28902114306E0D903090C8D
:100A0000DF0701D0491C89B2890231806178002951
:100A100002D0012918D01FE001685026765A7118BB
:100A20002678F60075194D193E2B06D9D902090C06
:100A3000DB06D8D1491E89B2D5E7D903090CDA07FC
:100A4000D4D0491C89B2D1E701685022525A5118BA
:100A50002278D20052198B52016820788200885A7D
:100A6000064B184001231B0358405B005840044BC1
:100A7000184388520020F0BD060400008FBF00001C
:100A800080800000F0B50246FF32E132137A012B7C
:100A90000BD001244F06CB097F0E1472002B06D019
:100AA0001C237B431B18283306E00220F0BD1C23C7
:100AB0004B431B18FF3309339C701F70CE095E70C7
:100AC000012424031025114B002F0BD04906C90D1A
:100AD000002E10D00468605A0D4E30406840184314
:100AE000605210E0016808880A4E3040604068405B
:100AF0001843088007E00568685A064E303E3040CB
:100B000060401843685200201072F0BD80800000E1
:100B1000BF8F0000BFBF0000F0B506461D46480667
:100B2000400E1C2343439C19E563A2630022226408
:100B30000123283463702070E0682B46854203D976
:100B40000546181A606100E06261A07A2A4F002809
:100B500010D0227830689200825A49065206890DD8
:100B6000002A16DA5022125A10183A1D89184552D6
:100B7000228914E0ABB2A2882169306800F007FF37
:100B800030685021095A08182178C900C9194552FE
:100B900020E05022125A1018C9194552E288ABB20F
:100BA0002169306800F0F3FE61781448002902D012
:100BB000012907D00EE0217832688B00D15A01401C
:100BC0000F4805E0217832688B00D15A01400D486A
:100BD0000143D152207831688200885A074B303364
:100BE00018401023584020235840054B403B1843E1
:100BF00088520020F0BD0000020400008F8F00002A
:100C0000C080000080C0000070B50446006840301D
:100C10008088C00B02D0204600F006FD20684030DE
:100C2000818849050AD58188334A11408180204650
:100C300000F0DAF80021204600F008F92068403082
:100C40008188490403D581882C4A1140818020681D
:100C500040308188890403D58188294A11408180E8
:100C60002068403081880425C904002910DA0188F1
:100C7000A9430180BD202168000240310880204640
:100C800000F0C6F82068403081881E4A11408180FB
:100C9000206840308188090517D581881A4A11409B
:100CA000818020684030018808221143018020683B
:100CB0004030018829430180206840308088C0434B
:100CC000C00402D5204600F0EBF82068403081884F
:100CD000890506D581880D4A11408180204600F0A3
:100CE000ADF8206840308188C90503D58188084A5D
:100CF0001140818070BD0000FFFB0000FFBF0000BD
:100D0000FFDF0000FFEF0000FFF70000FFFD000025
:100D1000FFFE0000F8B500270446002807D026464D
:100D2000FF36E136707A0025002802D005E0012068
:100D3000F8BD3572204600F03BF8032070720121A7
:100D40000BE01C20784302191046203041720772D4
:100D5000C572556395637F1CD5636068B842F0D84F
:100D600000200BE01C2242431219FF32013255725F
:100D70001072D57255619561401CD56162688242DE
:100D8000F0D820684030018020684030058020681D
:100D900040308580206840300582BF2022680002F4
:100DA000403210802034257171720020F8BD00009F
:100DB00008B500680A49884210D10A48C269012171
:100DC000C9050A43C261C06900220840009011466B
:100DD0001F20FFF723FB1F20FFF716FB08BD0000B5
:100DE000005C00400010024070B504468068012598
:100DF000022801D0FFF7FFF9FF34FF3402342946FF
:100E0000E06901F086F9E06901F04BF970BD00007E
:100E100010B504468069002806D0074801690622FB
:100E20009143016100F0CCFDFF34FF340234E069EE
:100E300001F05AF910BD000000ED00E0FF3010B5E0
:100E4000FF300230C06901F055F910BD0246FF3293
:100E5000E132137A012B08D001231372002906D046
:100E60002030017100201072704702207047006826
:100E7000802140308181F5E710B5872189000A582B
:100E80000146FF31ED31104601F050F910BD006808
:100E90004030018B0122D2031143018300207047AF
:100EA00010B50446FF30FF300230C06901F081F90F
:100EB000A069002804D0034801690622114301619A
:100EC00010BD000000ED00E0F8B505460068394CA3
:100ED000C00352D5E0690026C00007D4E1692004B0
:100EE0000143E161E1690140012600913248016856
:100EF000C90510D40168821511430160FFF73AFA61
:100F0000074604E0FFF736FAC01B642824D82A48B5
:100F10000068C005F6D5206A03273F02384020D07C
:100F20006968394081421CD0206A226AB843012195
:100F300009040A432262226A8A4322622062C007AD
:100F40000FD0FFF717FA009008E0FFF713FA0099A7
:100F5000411A1A48814201D90320F8BD206A80074E
:100F6000F3D5206A6968B84308432062002E04D094
:100F7000E169012000078143E1612878C00705D0BD
:100F8000206BA968800880000843206328788006C9
:100F900005D5206B10218843E96808432063286841
:100FA000800305D5206B802188432969084320638D
:100FB0000020F8BD001002400070004088130000BF
:100FC000F8B5054644480E460068C007C00FB04259
:100FD0000AD241480168490849003143016000686C
:100FE000C007C00FB0425CD128783C4C800705D5C3
:100FF0006068F0218843A968084360602878C007CA
:101000003FD06868012813D02168022813D08907CF
:10101000002946DA61688908890001436160FFF7A9
:10102000A9F96968074601290DD0022917D024E0E3
:1010300021688903ECE78901EAE7FFF79BF9C11B07
:101040002748814217D860680007800F0128F4D133
:1010500017E0FFF78FF9C11B214881420BD8606868
:101060000007800F0228F4D10BE0FFF783F9C11BC2
:101070001B48814201D90320F8BD60680007800F3A
:10108000F3D115480168C907C90FB1420BD90168EE
:1010900049084900314301600068C007C00FB042F1
:1010A00001D00120F8BD2878400706D560680721E7
:1010B00009028843E9680843606000F01DF8616830
:1010C000084A0906090F515CC8400749086000201A
:1010D000FFF76EF90020F8BD00200240001002402A
:1010E00088130000002600087400002001480068F2
:1010F000704700007400002010B511A30FCB88B01A
:101100006C460FC412A30FCB0FC415494A680C20BC
:10111000134603401348042B0FD0082B0DD1930224
:101120001B0F6C46E45CC96A04AB0907090FD203C4
:10113000595C920FFEF7FAFF604308B010BD000043
:1011400002030405060708090A0B0C0D0E0F101008
:101150000102030405060708090A0B0C0D0E0F1007
:101160000010024000127A00FEB504460078D24D0D
:10117000C00749D068680007800F012820D0686840
:101180000007800F022804D16868C003800F02287E
:1011900016D0012062680004012A18D08100002ABC
:1011A00001D0052A17D02A6882432A60286888431C
:1011B0002860606800281BD0FFF7DCF8064613E0C3
:1011C0002868800320D56068002876D01CE0296854
:1011D00001432960EDE72A680A432A60F7E7FFF731
:1011E000C9F8801B642869D828688003F7D50BE00C
:1011F000FFF7C0F8064604E0FFF7BCF8801B642840
:10120000F1D828688003F7D42078012680070028C9
:101210003DDA68680007800F13D068680007800F08
:10122000022804D16868C003800F012809D0E06853
:10123000002828681CD030432860FFF79BF8074639
:101240000BE0286880070BD5E068012835D107E05E
:10125000FFF790F8C01B0228C5D828688007F7D58B
:101260002868F82188432169C900084328600EE0F6
:10127000400840002860FFF77DF8074604E0FFF7CC
:1012800079F8C01B0228AED828688007F7D42078E8
:10129000000723D5E0690028686A10D030436862EF
:1012A000FFF768F8074604E0FFF764F8C01B022860
:1012B00099D8686A8007F7D510E0FAE0A4E0400802
:1012C00040006862FFF756F8074604E0FFF752F85F
:1012D000C01B022887D8686A8007F7D420780427C3
:1012E0004007002860DA00200190E869C00008D4B7
:1012F000E969B8060143E961E9690140012000910B
:1013000001906E480168C90511D401688215114326
:101310000160FFF72FF8009005E0FFF72BF8009928
:10132000401A642870D865480068C005F5D5A068E3
:1013300001280AD0002801D0052810D0286A4008CA
:1013400040002862286AB84301E0286A30432862D6
:10135000A068002812D0FFF70DF800900AE0286A74
:1013600038432862F1E7FFF705F80099411A54481D
:10137000814249D8286A8007F5D50DE0FEF7FAFFCB
:10138000009006E0FEF7F6FF0099411A4C488142B2
:101390003AD8286A8007F5D40198002804D0E96972
:1013A000012000078143E9612078C00635D56069D6
:1013B00001280CD0401D686B23D038436863686BEC
:1013C000400840006863FEF7D5FF064622E0686BE0
:1013D00038436863686B30436863FEF7CBFF0646AB
:1013E00004E0FEF7C7FF801B02285BD8686B80070C
:1013F000F7D5686BF8218843A169C9000843686381
:101400000BE0B8436863F4E74CE0FEF7B3FF801BE2
:10141000022847D8686B8007F7D4206A002846D096
:1014200069680907890F022943D001263606022878
:10143000286805D0B0432860FEF79CFF044633E0DF
:10144000B0432860FEF796FF074604E0FEF792FFE0
:10145000C01B022826D828688001F7D4E86AE16A10
:10146000000900010843E862616AA06A08436968EC
:101470007B22D20391430843686028683043286088
:10148000FEF778FF044604E0FEF774FF001B022815
:1014900008D828688001F7D509E0FEF76BFF001B2C
:1014A000022801D90320FEBD28688001F5D4002060
:1014B000FEBD0120FEBD0000001002400070004093
:1014C00088130000094910B5401E884201D9012047
:1014D00010BD074C60610321081F00F083F8002055
:1014E000A06107202061002010BD0000FFFFFF0069
:1014F00000E000E0FEE770B500231D460EE0040F9B
:101500000A2C02D25E00303401E05E0037348C5584
:101510005C00641800015B1C6570DBB29342EED383
:1015200070BD000070B586B014216846FEF71BFE42
:1015300019484269012189050A43426142690A400A
:101540000592426949110A43426142690A40059283
:10155000426949000A4342614069104E08400590C3
:10156000002202213046FEF7FEFE32200024012533
:101570006A4631C209206946C006FEF74BFE0220CA
:101580000090032003900195029469463046FEF7CF
:1015900041FE06B070BD000000100240000400488B
:1015A00010B500220B490C4800F05AFC002801D06D
:1015B000FEF721FE0949084800F021FE002801D06D
:1015C000FEF719FE044800F06BFE002801D0FEF77C
:1015D00012FE10BD200000204C0100207C000020E5
:1015E000704700008307FF22DB0E9A408907090E2F
:1015F000994000280BDA0007000F083883080848D4
:101600009B001818C36993430B43C3617047830859
:1016100004489B001B1818689043084318607047E3
:1016200000ED00E000E400E0F0B585B004460021E4
:101630006846818020462030029079E19A89170718
:101640003F0F24D0BE00815B99809988090470D532
:10165000815BBF4A114081531C2078430519FF3537
:101660000935A87A002820687ED029788A00825A15
:1016700052047AD55022125ACB00B6491218591882
:10168000515A8905890D009170D0EA88C1E09A8984
:10169000D2062BD40288B0490A4002802068254631
:1016A000283501464030008A41182878C200A948F0
:1016B0001018085A8005800D2064A16B0818A063DB
:1016C00000212046FEF7CBFE029800790028B4D016
:1016D00068690028B1D10298007980210843216807
:1016E0004031888102980021017121E12546FF35B2
:1016F000038809356A469380928812051AD5098AAB
:1017000009182878C2009348001D1018085A294665
:1017100083059B0DAB61AA88E431206800F022F9B3
:10172000206801888A4A114001802046FFF7A4FB07
:10173000FEE095E0694689880904D6D50188844A87
:101740001140018020685021095A824E08182978DA
:10175000361DC9008919405A83059B0DAB610CD019
:10176000AA882969206802E033E045E055E000F0EE
:10177000F9F8A96928694018286100212046FEF778
:101780007AFE20685021095A08188219E8683E2814
:101790000AD9C102090CC00601D1491E89B28802CA
:1017A0000121C903084306E0C103090CC00701D0A9
:1017B000491C89B28802108021680888674A104055
:1017C00001221203504052005040654A10430880E5
:1017D000AEE05021095A0A182978CB005D49091D4D
:1017E0005918515A8905890D009121D0AA88296973
:1017F000009B00F0B7F81BE05022CB00125A55496D
:101800001218091D5918515A8905890D009104D0E3
:101810002A892969009B00F0A5F8287822688000B1
:10182000115A4D4B803319404D4B403319431152DF
:10183000A96900980818A8612869009942182A61C6
:101840006B69002B03D0E9680098814204D929789C
:101850002046FEF710FE03E029782046FFF792F8B5
:1018600068468088000663D51C20474320683D19E0
:10187000815B394A114081532835A87A00282068B5
:1018800011D029788A00825A52061ED55022125A47
:10189000C90012182F480818105A83059B0DAB6118
:1018A00024D0EA881EE05021095A09182878C2007D
:1018B00028481018085A83059B0DAB6121D0AA88CF
:1018C0002969206800F063F81BE05022125AC90011
:1018D00012182048001D0818105A83059B0DAB6193
:1018E00004D02A892969206800F051F829782068F5
:1018F0008A00815A184B80331940184BF133194331
:101900008152206802464030018A28788A1811499D
:10191000C0004018105A8005800DA86129690A1876
:101920002A616B692978002B20460DD0FFF7F4F867
:101930002068014640318A886B469A81120400D59E
:101940007CE6002005B0F0BDFEF789FDF0E7000061
:101950008F0F0000020400000F8F00008FBF0000F7
:1019600080800000101810B5012292025C088018D7
:10197000002C07D002880A70120A4A70801C891C49
:10198000641EF7D1DA0701D00078087010BD101876
:1019900001225B1C920210B55B088018002B08D056
:1019A0004A780C78120222430280801C891C5B1E3C
:1019B000F6D110BD7047704710B5FEF7E1FC10BDC1
:1019C00030B595B030216846FEF7CDFB00240C946D
:1019D0000D940E94142110A80F94FEF7C4FB01205F
:1019E0000190009000040990000102250A900895DA
:1019F0000B946846FFF7B8FB07200C900E9401216A
:101A00000D950F940CA8FFF7DBFA280410908020A6
:101A1000149010A8FFF758FA15B030BD15480168AA
:101A20000122114301604168134A1140416001687D
:101A3000124A114001600168012292049143016041
:101A400041683F22120491434160C16A09090901BA
:101A5000C162016BFF22943291430163016B8022CA
:101A600011430163416B49084900416300218160D2
:101A700070470000001002400CB8FF08FFFFF6FEA0
:101A800010B585229200125852689047002010BD70
:101A9000134610B50A46002100F0F9FA002010BDE7
:101AA000134610B50A46002100F08BFB002010BD44
:101AB00010B50446802100F068FB0021204600F0AC
:101AC00064FB10BD10B5FF210522F5310A5000233B
:101AD0001A46194600F0DBFA002010BD10B5FF23AE
:101AE0000224F5331C5082611346C2610A4600216C
:101AF00000F067FB002010BD10B5FF210422F53176
:101B00000A5000231A46194600F05BFB002010BD66
:101B100010B50A46024903A000F0D2F8004810BDF3
:101B2000A405002048494420436F6E6669670000A1
:101B300012200880004870474000002010B50A4677
:101B4000024903A000F0BCF8004810BDA405002025
:101B500048494420496E74657266616365000000FF
:101B600004200880004870473C00002010B50A4659
:101B7000024903A000F0A4F8004810BDA40500200D
:101B800054796E65742E65750000000010B50A4624
:101B9000024903A000F094F8004810BDA4050020FD
:101BA00056464F204B6E6F620000000010B51A20A1
:101BB00008800948046BC16A406B081809D00822E4
:101BC0000649FFF798FC0549042210312046FFF72B
:101BD00092FC0248801E10BD80F7FF1F56000020B7
:101BE000F8B50D4604464988FF300A0AFF30023036
:101BF000130000F071FC084905091649493E4649A1
:101C00000069237C02682AE0217C022640690029C1
:101C100005D0C16A684688470146467040E0816A3F
:101C2000F8E7C9B20B0000F057FC0604080F1317C1
:101C30001E2F0069227C436802E00069227C8368D1
:101C400069461046984712E00069227CC368F7E7AE
:101C50000069227C0369F3E70069237C42696946D5
:101C60001846904703E00069227C8369E8E7014653
:101C700016E0217C002907D14069416B68468847FE
:101C8000F5E7217C002904D029462046FFF710FF04
:101C9000F8BD4069016B68468847072201464270DB
:101CA000684600880028F3D0EA88002AF0D08242F3
:101CB00000D90246684602802046FFF70FFFF8BDB4
:101CC00070B5002300281CD00446002502E06D1CDE
:101CD000EDB2641C2678002EF9D16C00A41C14808F
:101CE000CC5403225B1CCA5400245B1C06E0CA547B
:101CF0005B1CDAB28C54521CD3B2401C0278002A0E
:101D0000F5D170BD01460020002904D0012901D081
:101D1000022901D00220704701207047FF300021C6
:101D2000FF300230806901730846704710B50446E1
:101D3000812100F0B8F8FF34FF340234A069002894
:101D400003D000F0BBFB0020A061002010BD00000C
:101D50002221018000487047B40000200A21018040
:101D600000487047E400002070B5054600240423B5
:101D70000322812100F07EF9102000F0A1FBFF3545
:101D8000FF350235A861002803D0002101732046E9
:101D900070BD0124FBE710B51346FF244322FD3438
:101DA000D200245C1258032C08D1147B002C05D1DE
:101DB000012414730A46812100F003FA002010BDAB
:101DC00070B543230022DB000D781B5860261446B3
:101DD00035401BD0202D3ED14A78022A13D0032A49
:101DE0000AD00A2A0BD00B2A03D0FFF761FE02208B
:101DF00070BD887818602EE00122194622E04888DC
:101E0000000A586027E00122191D1BE04D78062DBD
:101E100004D00A2D19D00B2D1DD11AE04B881B0AB6
:101E2000222B02D0212B06D00BE0CA885B2A00D9D6
:101E30005B220A4C05E0094CCA88183C092A00D9E3
:101E400009222146FFF74AFE05E001221946083122
:101E5000F8E788789860002070BD0000F00000204E
:101E600010B5002813D0C31DFF33FA335C69002C72
:101E700001D000245C61002900D01961FF210123F9
:101E8000FD310B54027000F0ADF8002010BD0220AF
:101E900010BDFF3010B5FF300230006AFEF7B4FB12
:101EA000FFF730FF10BDFF3010B5FF300230006A81
:101EB000FEF7F0FAFFF726FF10BDFEB50446FF302F
:101EC000E51DE130FF35FA3513460190002908D0B1
:101ED00068694269002A49D00198007F032843D0ED
:101EE00044E02646FF3681362046716F14300229C1
:101EF00034D1C26881680092914207D9891A816001
:101F00008AB219462046FFF7CBFD13E04068114620
:101F10000746FEF70BF9002913D10098874210D32A
:101F2000B06F87420DD2002211462046FFF7B8FD60
:101F30000020B06700231A461946204600F0A7F893
:101F40000CE06869C168002905D00198007F03286A
:101F500001D1204688472046FFF7B4FD28780128A4
:101F600004D10020287001E0204690470020FEBDEB
:101F700070B50546FF35E1352B462033164604463D
:101F8000002907D058698269002A29D0287F0328B0
:101F900024D025E0FF21F531E01D0959FD3003294A
:101FA0001ED18268C1688A420BD9511A8160C0680B
:101FB000814200D301468AB231462046FFF768FDD0
:101FC0000EE058690169002904D0287F032801D157
:101FD000204688472046FFF78FFD01E020469047C6
:101FE000002070BD10B51749C41DC861FF341649E3
:101FF000FA34164821620860082048600220886090
:10200000086100208861C86108620846FEF782FE08
:10201000002801D0FEF7EFF8002218231146206AAD
:10202000FEF700FA582300228021206AFEF7FAF911
:10203000FF23013300228121206AFEF7F3F90020FB
:1020400010BD00008405002084030020005C0040D7
:10205000FF30CA09FF3049060230490E1C23006ACE
:1020600059430818002A01D0203001E0FF30013028
:10207000807A704710B5FF301C46FF30023013469F
:10208000006A2246FEF71CFBFFF73CFE10BDFF3046
:1020900010B5FF300230006AFEF774FCFFF732FE25
:1020A00010BD70B50022044640231146FFF7E2FF41
:1020B0004025FF20113005512B460022802120466B
:1020C000FFF7D8FFFF200121FD3025620155E01DFB
:1020D000FF30FA308169002904D0406921794268D3
:1020E00020469047002070BDFF30E130417F0177EE
:1020F0000020704710B5FF21FD31095C032906D18E
:10210000852189000958C969002900D08847002025
:1021100010BD017400207047FF3010B5FF30023051
:10212000006AFEF793FEFFF7EDFD10BD70B50446A3
:102130004120C0002018054600F04DF82146FF312F
:1021400081310122084680304A67C2898A67007A55
:10215000C106C90E0AD001290DD0022910D0C1092B
:10216000C901204600F011F8002070BD2946204624
:1021700000F09BF8F8E72946204600F082F9F3E7E3
:102180002946204600F008F9EEE7FF3010B5FF3091
:102190000230006AFEF776FCFFF7B4FD10BDFF3099
:1021A00010B5FF300230006AFEF771FEFFF7AAFD9E
:1021B00010BDFF30E130017F41770421017700201D
:1021C0007047FF3010B5FF300230006AFEF7A4FC04
:1021D000FFF798FD10BD0A7802704A784270CB78FC
:1021E0008A781B02D21842804B790A791B02D218D6
:1021F00082808A79C97909025118C18070470246E4
:102200000020002904D0FF32FF32023251617047B2
:102210000220704710B58522920012580224002A2D
:1022200004D012689047002800D10024204610BD39
:1022300070B50E468978194D04462970012904D9D4
:1022400031462046FFF734FC70BD2046FF30E130B8
:10225000027F022A15D0032AF2D1002917D0606824
:1022600088420AD0C1B22046FFF70AFC2978616093
:102270002046FFF7CFFF0228E2D02046FFF73CFCC4
:1022800070BD0029F9D0032261600277F0E70222D5
:10229000027720466160FFF7F3FBEEE7780000204D
:1022A00010B5FFF77CFF002010BDF8B500220092AA
:1022B000C61DFF364C781746FA3632460125203ABD
:1022C000230000F009F90A3C564150410906412B10
:1022D0002841FFF785FC5DE004468888002818D176
:1022E000C888002815D1887817464606107F760ED4
:1022F00003280ED0BE7731462046FFF70DFF20465B
:10230000FFF7FAFB002E02D00220387742E03D773B
:1023100040E0204618E0FFF78BFF3BE0CB88012B25
:1023200012D1127F022A02D0032A0DD104E0012229
:1023300001460831876013E00122011D10E0127F81
:10234000022A04D0032A02D0FFF7B2FB22E0C560C4
:102350007168002901D00321C160014602220C31BD
:10236000FFF7BCFB16E004464888012812D17560CF
:1023700009E00446107F022801D00328C9D148880B
:10238000012807D17760706982682046904720460F
:10239000FFF7B2FB0098F8BDF8B504460D46287863
:1023A000E61D4006FF3600270979800FFA3601281E
:1023B00009D06A7830462038002A38D0012A1ED049
:1023C000032A3DD106E0706929468268204690477D
:1023D0000020F8BD007F022817D003282CD1688880
:1023E000002806D1002904D0802902D02046FFF71A
:1023F000CCFE7069294682682046904713E0007F32
:10240000022802D0032817D104E0002918D080291F
:102410001AD115E06888002812D1480603D020465A
:10242000FFF737FDE5E72046FFF766FB08E0007F92
:10243000022807D003280BD029462046FFF738FB97
:102440003846F8BD4806FBD02046FFF79EFEF7E76A
:10245000C80904D04806400D0519143504E04806A3
:10246000400D0519FF3505352046FFF7F1FD002821
:1024700000D001202860022229462046FFF72EFBCB
:10248000DEE770B50446FF30E130007F0D460328DB
:102490000FD1287901280CD8852080000059826846
:1024A00020469047E888002806D12046FFF724FB05
:1024B00002E02046FFF7FCFA002070BD70470000E4
:1024C000004870477003002010B50248FEF79CFBDF
:1024D00010BD00008403002030B47446641E2578CB
:1024E000641CAB4200D21D46635D5B00E31830BC48
:1024F000184702E008C8121F08C1002AFAD1704725
:102500007047002001E001C1121F002AFBD1704773
:10251000FDF73EFF0925ED0610212846FDF71EFFB9
:10252000344CE060FFF74CFA204601270221676037
:102530000646017018363770FEF7F4FFFFF730F8E3
:10254000012202212C48FDF70EFF20212846FDF72D
:1025500005FF00281CD00020606110212846FDF7EF
:10256000FDFEA060E16888420FD002212846FDF7F9
:10257000F5FEA1688842207900D140421D493071A2
:10258000052218311D48FFF706FCA068E060DCE773
:102590006069002803D1FDF7EDFE67612061606886
:1025A000012822D0052822D06760FDF7E3FE2169CB
:1025B000401A7D21C900884213D90E48202141705C
:1025C000014602220D48FFF7E6FB6420FDF714FEEA
:1025D00008490020487002220848FFF7DCFB002071
:1025E0006061C820FDF708FEB7E7052000E00A207B
:1025F0006060DAE700000020000400484C01002081
:1026000000000000000000000102030406070809A2
:1026100030260008000000204C010000A001000846
:10262000042700084C0100205C0A00000225000875
:10263000012013311B1B0861041A6D041A8D041A42
:10264000AD041A11041A3D041704030904120132DF
:1026500002164083042B57260201020301031F1AAE
:102660000353127A13691D1B082D041AC104819AA1
:102670001D0C811A511469041A5D041409022213F5
:10268000010125E03209042A016D15092111011407
:1026900001225B1607058103049A0A12314B0A06D0
:1026A000A4199B11100A05010902A1010901A11039
:1026B0000A850105091901290315180F250195033C
:1026C00075018102950175058101221814300931C7
:1026D00009381581257F750895038106C0C0050C52
:1026E000322E018502050C2E10187501950809B5CA
:1026F00009B609B709B809CD09E209E909EA810271
:04270000C000000015
:04000005080000C12E
:00000001FF
